 CallerAccessTest

 Timestamp is 7203bd00 (reproducible build file hash)

 Preferred load address is 0000000140000000

 Start         Length     Name                   Class
 0001:00000000 000012a0H .text$mn                CODE
 0001:000012a0 00000036H .text$mn$00             CODE
 0001:000012d6 00000036H .text$x                 CODE
 0002:00000000 000001a0H .idata$5                DATA
 0002:000001a0 00000038H .00cfg                  DATA
 0002:000001d8 00000008H .CRT$XCA                DATA
 0002:000001e0 00000008H .CRT$XCAA               DATA
 0002:000001e8 00000008H .CRT$XCZ                DATA
 0002:000001f0 00000008H .CRT$XIA                DATA
 0002:000001f8 00000008H .CRT$XIAA               DATA
 0002:00000200 00000008H .CRT$XIAC               DATA
 0002:00000208 00000008H .CRT$XIZ                DATA
 0002:00000210 00000008H .CRT$XPA                DATA
 0002:00000218 00000008H .CRT$XPZ                DATA
 0002:00000220 00000008H .CRT$XTA                DATA
 0002:00000228 00000008H .CRT$XTZ                DATA
 0002:00000230 00000000H .gehcont$y              DATA
 0002:00000230 00000000H .gfids$y                DATA
 0002:00000230 000004d0H .rdata                  DATA
 0002:00000700 00000000H .rdata$CastGuardVftablesA DATA
 0002:00000700 00000000H .rdata$CastGuardVftablesC DATA
 0002:00000700 00000048H .rdata$voltmd           DATA
 0002:00000748 000002c8H .rdata$zzzdbg           DATA
 0002:00000a10 00000008H .rtc$IAA                DATA
 0002:00000a18 00000008H .rtc$IZZ                DATA
 0002:00000a20 00000008H .rtc$TAA                DATA
 0002:00000a28 00000008H .rtc$TZZ                DATA
 0002:00000a30 00000104H .xdata                  DATA
 0002:00000b34 00000000H .edata                  DATA
 0002:00000b34 000000a0H .idata$2                DATA
 0002:00000bd4 00000014H .idata$3                DATA
 0002:00000be8 000001a0H .idata$4                DATA
 0002:00000d88 00000454H .idata$6                DATA
 0003:00000000 00000040H .data                   DATA
 0003:00000040 000000c8H .bss                    DATA
 0004:00000000 0000018cH .pdata                  DATA

  Address         Publics by Value              Rva+Base               Lib:Object

 0000:00000000       __AbsoluteZero             0000000000000000     <absolute>
 0000:00000000       ___safe_se_handler_count   0000000000000000     <absolute>
 0000:00000000       ___safe_se_handler_table   0000000000000000     <absolute>
 0000:00000000       __arm64x_extra_rfe_table   0000000000000000     <absolute>
 0000:00000000       __arm64x_extra_rfe_table_size 0000000000000000     <absolute>
 0000:00000000       __arm64x_native_entrypoint 0000000000000000     <absolute>
 0000:00000000       __arm64x_redirection_metadata 0000000000000000     <absolute>
 0000:00000000       __arm64x_redirection_metadata_count 0000000000000000     <absolute>
 0000:00000000       __dynamic_value_reloc_table 0000000000000000     <absolute>
 0000:00000000       __enclave_config           0000000000000000     <absolute>
 0000:00000000       __guard_check_icall_a64n_fptr 0000000000000000     <absolute>
 0000:00000000       __guard_eh_cont_count      0000000000000000     <absolute>
 0000:00000000       __guard_eh_cont_table      0000000000000000     <absolute>
 0000:00000000       __guard_fids_count         0000000000000000     <absolute>
 0000:00000000       __guard_fids_table         0000000000000000     <absolute>
 0000:00000000       __guard_iat_count          0000000000000000     <absolute>
 0000:00000000       __guard_iat_table          0000000000000000     <absolute>
 0000:00000000       __guard_longjmp_count      0000000000000000     <absolute>
 0000:00000000       __guard_longjmp_table      0000000000000000     <absolute>
 0000:00000000       __hybrid_auxiliary_iat     0000000000000000     <absolute>
 0000:00000000       __hybrid_auxiliary_iat_copy 0000000000000000     <absolute>
 0000:00000000       __hybrid_code_map          0000000000000000     <absolute>
 0000:00000000       __hybrid_code_map_count    0000000000000000     <absolute>
 0000:00000000       __x64_code_ranges_to_entry_points 0000000000000000     <absolute>
 0000:00000000       __x64_code_ranges_to_entry_points_count 0000000000000000     <absolute>
 0000:00000100       __guard_flags              0000000000000100     <absolute>
 0000:00000000       __ImageBase                0000000140000000     <linker-defined>
 0001:00000000       __local_stdio_printf_options 0000000140001000 f i exeCallerAccessTest.obj
 0001:00000008       checkAccess                0000000140001008 f   exeCallerAccessTest.obj
 0001:00000110       checkAndClearIllegalAccessExceptionThrown 0000000140001110 f   exeCallerAccessTest.obj
 0001:00000158       getField                   0000000140001158 f   exeCallerAccessTest.obj
 0001:00000244       main                       0000000140001244 f   exeCallerAccessTest.obj
 0001:0000025c       printf                     000000014000125c f i exeCallerAccessTest.obj
 0001:000005d4       setAccessible              00000001400015d4 f   exeCallerAccessTest.obj
 0001:000006c4       trySetAccessible           00000001400016c4 f   exeCallerAccessTest.obj
 0001:00000a28       mainCRTStartup             0000000140001a28 f   MSVCRT:exe_main.obj
 0001:00000a3c       __scrt_acquire_startup_lock 0000000140001a3c f   MSVCRT:utility.obj
 0001:00000a78       __scrt_initialize_crt      0000000140001a78 f   MSVCRT:utility.obj
 0001:00000ac4       __scrt_initialize_onexit_tables 0000000140001ac4 f   MSVCRT:utility.obj
 0001:00000b50       __scrt_is_nonwritable_in_current_image 0000000140001b50 f   MSVCRT:utility.obj
 0001:00000be8       __scrt_release_startup_lock 0000000140001be8 f   MSVCRT:utility.obj
 0001:00000c0c       __scrt_uninitialize_crt    0000000140001c0c f   MSVCRT:utility.obj
 0001:00000c38       _onexit                    0000000140001c38 f   MSVCRT:utility.obj
 0001:00000c74       atexit                     0000000140001c74 f   MSVCRT:utility.obj
 0001:00000c8c       __security_init_cookie     0000000140001c8c f   MSVCRT:gs_support.obj
 0001:00000d38       __scrt_exe_initialize_mta  0000000140001d38 f   MSVCRT:utility_desktop.obj
 0001:00000d38       __scrt_initialize_winrt    0000000140001d38 f   MSVCRT:utility_desktop.obj
 0001:00000d38       __scrt_stub_for_initialize_mta 0000000140001d38 f   MSVCRT:utility_desktop.obj
 0001:00000d38       _get_startup_commit_mode   0000000140001d38 f   MSVCRT:commit_mode.obj
 0001:00000d38       _get_startup_new_mode      0000000140001d38 f   MSVCRT:new_mode.obj
 0001:00000d38       _get_startup_thread_locale_mode 0000000140001d38 f   MSVCRT:thread_locale.obj
 0001:00000d38       _matherr                   0000000140001d38 f   MSVCRT:matherr.obj
 0001:00000d3c       _get_startup_argv_mode     0000000140001d3c f   MSVCRT:argv_mode.obj
 0001:00000d44       _get_startup_file_mode     0000000140001d44 f   MSVCRT:file_mode.obj
 0001:00000d4c       ?__scrt_initialize_type_info@@YAXXZ 0000000140001d4c f   MSVCRT:tncleanup.obj
 0001:00000d5c       __acrt_initialize          0000000140001d5c f   MSVCRT:ucrt_stubs.obj
 0001:00000d5c       __acrt_uninitialize        0000000140001d5c f   MSVCRT:ucrt_stubs.obj
 0001:00000d5c       __scrt_stub_for_acrt_initialize 0000000140001d5c f   MSVCRT:ucrt_stubs.obj
 0001:00000d5c       __scrt_stub_for_acrt_uninitialize 0000000140001d5c f   MSVCRT:ucrt_stubs.obj
 0001:00000d5c       __vcrt_initialize          0000000140001d5c f   MSVCRT:ucrt_stubs.obj
 0001:00000d5c       __vcrt_uninitialize        0000000140001d5c f   MSVCRT:ucrt_stubs.obj
 0001:00000d5c       _should_initialize_environment 0000000140001d5c f   MSVCRT:env_mode.obj
 0001:00000d60       _guard_check_icall_nop     0000000140001d60 f   MSVCRT:guard_support.obj
 0001:00000d60       _initialize_denormal_control 0000000140001d60 f   MSVCRT:denormal_control.obj
 0001:00000d60       _initialize_invalid_parameter_handler 0000000140001d60 f   MSVCRT:invalid_parameter_handler.obj
 0001:00000d64       __local_stdio_scanf_options 0000000140001d64 f i MSVCRT:default_local_stdio_options.obj
 0001:00000d6c       __scrt_initialize_default_local_stdio_options 0000000140001d6c f   MSVCRT:default_local_stdio_options.obj
 0001:00000d88       __scrt_is_user_matherr_present 0000000140001d88 f   MSVCRT:matherr_detection.obj
 0001:00000d94       __scrt_get_dyn_tls_init_callback 0000000140001d94 f   MSVCRT:dyn_tls_init.obj
 0001:00000d9c       __scrt_get_dyn_tls_dtor_callback 0000000140001d9c f   MSVCRT:dyn_tls_dtor.obj
 0001:00000da4       __crt_debugger_hook        0000000140001da4 f   MSVCRT:utility_desktop.obj
 0001:00000dac       __scrt_fastfail            0000000140001dac f   MSVCRT:utility_desktop.obj
 0001:00000ef8       __scrt_initialize_mta      0000000140001ef8 f   MSVCRT:utility_desktop.obj
 0001:00000f00       __scrt_is_managed_app      0000000140001f00 f   MSVCRT:utility_desktop.obj
 0001:00000f54       __scrt_set_unhandled_exception_filter 0000000140001f54 f   MSVCRT:utility_desktop.obj
 0001:00000f64       __scrt_unhandled_exception_filter 0000000140001f64 f   MSVCRT:utility_desktop.obj
 0001:00000fc0       _RTC_Initialize            0000000140001fc0 f   MSVCRT:initsect.obj
 0001:00000ffc       _RTC_Terminate             0000000140001ffc f   MSVCRT:initsect.obj
 0001:00001038       __isa_available_init       0000000140002038 f   MSVCRT:cpu_disp.obj
 0001:000011e4       __scrt_is_ucrt_dll_in_use  00000001400021e4 f   MSVCRT:ucrt_detection.obj
 0001:000011f0       __C_specific_handler       00000001400021f0 f   vcruntime:VCRUNTIME140.dll
 0001:000011f6       __current_exception        00000001400021f6 f   vcruntime:VCRUNTIME140.dll
 0001:000011fc       __current_exception_context 00000001400021fc f   vcruntime:VCRUNTIME140.dll
 0001:00001202       memset                     0000000140002202 f   vcruntime:VCRUNTIME140.dll
 0001:00001208       exit                       0000000140002208 f   ucrt:api-ms-win-crt-runtime-l1-1-0.dll
 0001:0000120e       _seh_filter_exe            000000014000220e f   ucrt:api-ms-win-crt-runtime-l1-1-0.dll
 0001:00001214       _set_app_type              0000000140002214 f   ucrt:api-ms-win-crt-runtime-l1-1-0.dll
 0001:0000121a       __setusermatherr           000000014000221a f   ucrt:api-ms-win-crt-math-l1-1-0.dll
 0001:00001220       _configure_narrow_argv     0000000140002220 f   ucrt:api-ms-win-crt-runtime-l1-1-0.dll
 0001:00001226       _initialize_narrow_environment 0000000140002226 f   ucrt:api-ms-win-crt-runtime-l1-1-0.dll
 0001:0000122c       _get_initial_narrow_environment 000000014000222c f   ucrt:api-ms-win-crt-runtime-l1-1-0.dll
 0001:00001232       _initterm                  0000000140002232 f   ucrt:api-ms-win-crt-runtime-l1-1-0.dll
 0001:00001238       _initterm_e                0000000140002238 f   ucrt:api-ms-win-crt-runtime-l1-1-0.dll
 0001:0000123e       _exit                      000000014000223e f   ucrt:api-ms-win-crt-runtime-l1-1-0.dll
 0001:00001244       _set_fmode                 0000000140002244 f   ucrt:api-ms-win-crt-stdio-l1-1-0.dll
 0001:0000124a       __p___argc                 000000014000224a f   ucrt:api-ms-win-crt-runtime-l1-1-0.dll
 0001:00001250       __p___argv                 0000000140002250 f   ucrt:api-ms-win-crt-runtime-l1-1-0.dll
 0001:00001256       _cexit                     0000000140002256 f   ucrt:api-ms-win-crt-runtime-l1-1-0.dll
 0001:0000125c       _c_exit                    000000014000225c f   ucrt:api-ms-win-crt-runtime-l1-1-0.dll
 0001:00001262       _register_thread_local_exe_atexit_callback 0000000140002262 f   ucrt:api-ms-win-crt-runtime-l1-1-0.dll
 0001:00001268       _configthreadlocale        0000000140002268 f   ucrt:api-ms-win-crt-locale-l1-1-0.dll
 0001:0000126e       _set_new_mode              000000014000226e f   ucrt:api-ms-win-crt-heap-l1-1-0.dll
 0001:00001274       __p__commode               0000000140002274 f   ucrt:api-ms-win-crt-stdio-l1-1-0.dll
 0001:0000127a       _initialize_onexit_table   000000014000227a f   ucrt:api-ms-win-crt-runtime-l1-1-0.dll
 0001:00001280       _register_onexit_function  0000000140002280 f   ucrt:api-ms-win-crt-runtime-l1-1-0.dll
 0001:00001286       _crt_atexit                0000000140002286 f   ucrt:api-ms-win-crt-runtime-l1-1-0.dll
 0001:0000128c       terminate                  000000014000228c f   ucrt:api-ms-win-crt-runtime-l1-1-0.dll
 0001:00001292       memcpy                     0000000140002292 f   vcruntime:VCRUNTIME140.dll
 0001:000012b0       _guard_dispatch_icall_nop  00000001400022b0 f   MSVCRT:guard_dispatch.obj
 0001:000012d0       _guard_xfg_dispatch_icall_nop 00000001400022d0 f   MSVCRT:guard_xfg_dispatch.obj
 0002:00000000       __imp_GetModuleHandleW     0000000140003000     kernel32:KERNEL32.dll
 0002:00000008       __imp_QueryPerformanceCounter 0000000140003008     kernel32:KERNEL32.dll
 0002:00000010       __imp_GetCurrentProcessId  0000000140003010     kernel32:KERNEL32.dll
 0002:00000018       __imp_GetCurrentThreadId   0000000140003018     kernel32:KERNEL32.dll
 0002:00000020       __imp_GetSystemTimeAsFileTime 0000000140003020     kernel32:KERNEL32.dll
 0002:00000028       __imp_InitializeSListHead  0000000140003028     kernel32:KERNEL32.dll
 0002:00000030       __imp_RtlCaptureContext    0000000140003030     kernel32:KERNEL32.dll
 0002:00000038       __imp_RtlLookupFunctionEntry 0000000140003038     kernel32:KERNEL32.dll
 0002:00000040       __imp_RtlVirtualUnwind     0000000140003040     kernel32:KERNEL32.dll
 0002:00000048       __imp_IsDebuggerPresent    0000000140003048     kernel32:KERNEL32.dll
 0002:00000050       __imp_UnhandledExceptionFilter 0000000140003050     kernel32:KERNEL32.dll
 0002:00000058       __imp_SetUnhandledExceptionFilter 0000000140003058     kernel32:KERNEL32.dll
 0002:00000060       __imp_IsProcessorFeaturePresent 0000000140003060     kernel32:KERNEL32.dll
 0002:00000068       \177KERNEL32_NULL_THUNK_DATA 0000000140003068     kernel32:KERNEL32.dll
 0002:00000070       __imp_memset               0000000140003070     vcruntime:VCRUNTIME140.dll
 0002:00000078       __imp_memcpy               0000000140003078     vcruntime:VCRUNTIME140.dll
 0002:00000080       __imp___C_specific_handler 0000000140003080     vcruntime:VCRUNTIME140.dll
 0002:00000088       __imp___current_exception  0000000140003088     vcruntime:VCRUNTIME140.dll
 0002:00000090       __imp___current_exception_context 0000000140003090     vcruntime:VCRUNTIME140.dll
 0002:00000098       \177VCRUNTIME140_NULL_THUNK_DATA 0000000140003098     vcruntime:VCRUNTIME140.dll
 0002:000000a0       __imp__set_new_mode        00000001400030a0     ucrt:api-ms-win-crt-heap-l1-1-0.dll
 0002:000000a8       \177api-ms-win-crt-heap-l1-1-0_NULL_THUNK_DATA 00000001400030a8     ucrt:api-ms-win-crt-heap-l1-1-0.dll
 0002:000000b0       __imp__configthreadlocale  00000001400030b0     ucrt:api-ms-win-crt-locale-l1-1-0.dll
 0002:000000b8       \177api-ms-win-crt-locale-l1-1-0_NULL_THUNK_DATA 00000001400030b8     ucrt:api-ms-win-crt-locale-l1-1-0.dll
 0002:000000c0       __imp___setusermatherr     00000001400030c0     ucrt:api-ms-win-crt-math-l1-1-0.dll
 0002:000000c8       \177api-ms-win-crt-math-l1-1-0_NULL_THUNK_DATA 00000001400030c8     ucrt:api-ms-win-crt-math-l1-1-0.dll
 0002:000000d0       __imp__seh_filter_exe      00000001400030d0     ucrt:api-ms-win-crt-runtime-l1-1-0.dll
 0002:000000d8       __imp__configure_narrow_argv 00000001400030d8     ucrt:api-ms-win-crt-runtime-l1-1-0.dll
 0002:000000e0       __imp__initialize_narrow_environment 00000001400030e0     ucrt:api-ms-win-crt-runtime-l1-1-0.dll
 0002:000000e8       __imp__get_initial_narrow_environment 00000001400030e8     ucrt:api-ms-win-crt-runtime-l1-1-0.dll
 0002:000000f0       __imp__initterm            00000001400030f0     ucrt:api-ms-win-crt-runtime-l1-1-0.dll
 0002:000000f8       __imp__initterm_e          00000001400030f8     ucrt:api-ms-win-crt-runtime-l1-1-0.dll
 0002:00000100       __imp__exit                0000000140003100     ucrt:api-ms-win-crt-runtime-l1-1-0.dll
 0002:00000108       __imp_terminate            0000000140003108     ucrt:api-ms-win-crt-runtime-l1-1-0.dll
 0002:00000110       __imp___p___argc           0000000140003110     ucrt:api-ms-win-crt-runtime-l1-1-0.dll
 0002:00000118       __imp___p___argv           0000000140003118     ucrt:api-ms-win-crt-runtime-l1-1-0.dll
 0002:00000120       __imp__cexit               0000000140003120     ucrt:api-ms-win-crt-runtime-l1-1-0.dll
 0002:00000128       __imp__c_exit              0000000140003128     ucrt:api-ms-win-crt-runtime-l1-1-0.dll
 0002:00000130       __imp__register_thread_local_exe_atexit_callback 0000000140003130     ucrt:api-ms-win-crt-runtime-l1-1-0.dll
 0002:00000138       __imp_exit                 0000000140003138     ucrt:api-ms-win-crt-runtime-l1-1-0.dll
 0002:00000140       __imp__crt_atexit          0000000140003140     ucrt:api-ms-win-crt-runtime-l1-1-0.dll
 0002:00000148       __imp__initialize_onexit_table 0000000140003148     ucrt:api-ms-win-crt-runtime-l1-1-0.dll
 0002:00000150       __imp__register_onexit_function 0000000140003150     ucrt:api-ms-win-crt-runtime-l1-1-0.dll
 0002:00000158       __imp__set_app_type        0000000140003158     ucrt:api-ms-win-crt-runtime-l1-1-0.dll
 0002:00000160       \177api-ms-win-crt-runtime-l1-1-0_NULL_THUNK_DATA 0000000140003160     ucrt:api-ms-win-crt-runtime-l1-1-0.dll
 0002:00000168       __imp___acrt_iob_func      0000000140003168     ucrt:api-ms-win-crt-stdio-l1-1-0.dll
 0002:00000170       __imp__set_fmode           0000000140003170     ucrt:api-ms-win-crt-stdio-l1-1-0.dll
 0002:00000178       __imp___stdio_common_vfprintf 0000000140003178     ucrt:api-ms-win-crt-stdio-l1-1-0.dll
 0002:00000180       __imp___p__commode         0000000140003180     ucrt:api-ms-win-crt-stdio-l1-1-0.dll
 0002:00000188       \177api-ms-win-crt-stdio-l1-1-0_NULL_THUNK_DATA 0000000140003188     ucrt:api-ms-win-crt-stdio-l1-1-0.dll
 0002:00000190       __imp_JNI_CreateJavaVM     0000000140003190     jvm:jvm.dll
 0002:00000198       \177jvm_NULL_THUNK_DATA    0000000140003198     jvm:jvm.dll
 0002:000001a0       __guard_check_icall_fptr   00000001400031a0     MSVCRT:guard_support.obj
 0002:000001a8       __guard_xfg_check_icall_fptr 00000001400031a8     MSVCRT:guard_support.obj
 0002:000001b0       __guard_dispatch_icall_fptr 00000001400031b0     MSVCRT:guard_support.obj
 0002:000001b8       __guard_xfg_dispatch_icall_fptr 00000001400031b8     MSVCRT:guard_support.obj
 0002:000001c0       __guard_xfg_table_dispatch_icall_fptr 00000001400031c0     MSVCRT:guard_support.obj
 0002:000001c8       __castguard_check_failure_os_handled_fptr 00000001400031c8     MSVCRT:guard_support.obj
 0002:000001d0       __guard_memcpy_fptr        00000001400031d0     vcruntime:softmemtag.obj
 0002:000001d8       __xc_a                     00000001400031d8     MSVCRT:initializers.obj
 0002:000001e8       __xc_z                     00000001400031e8     MSVCRT:initializers.obj
 0002:000001f0       __xi_a                     00000001400031f0     MSVCRT:initializers.obj
 0002:00000208       __xi_z                     0000000140003208     MSVCRT:initializers.obj
 0002:00000210       __xp_a                     0000000140003210     MSVCRT:initializers.obj
 0002:00000218       __xp_z                     0000000140003218     MSVCRT:initializers.obj
 0002:00000220       __xt_a                     0000000140003220     MSVCRT:initializers.obj
 0002:00000228       __xt_z                     0000000140003228     MSVCRT:initializers.obj
 0002:00000230       ??_C@_0BK@ELGCEAMJ@ERROR?3?5cannot?5create?5VM?4?6@ 0000000140003230     exeCallerAccessTest.obj
 0002:00000250       ??_C@_0BA@JJLOPNCP@java?1lang?1Class@ 0000000140003250     exeCallerAccessTest.obj
 0002:00000260       ??_C@_0CB@DKOJJLNI@java?1lang?1IllegalAccessExceptio@ 0000000140003260     exeCallerAccessTest.obj
 0002:00000288       ??_C@_0CG@NMJEAJOI@?$CILjava?1lang?1String?$DL?$CJLjava?1lang?1@ 0000000140003288     exeCallerAccessTest.obj
 0002:000002b0       ??_C@_07ILJBKILD@forName@  00000001400032b0     exeCallerAccessTest.obj
 0002:000002b8       ??_C@_0CO@ONFNEECC@?$CILjava?1lang?1String?$DL?$CJLjava?1lang?1@ 00000001400032b8     exeCallerAccessTest.obj
 0002:000002e8       ??_C@_08KAFPDKEA@getField@ 00000001400032e8     exeCallerAccessTest.obj
 0002:000002f8       ??_C@_0BI@HOMFJHGF@java?1lang?1reflect?1Field@ 00000001400032f8     exeCallerAccessTest.obj
 0002:00000310       ??_C@_0CH@JHKCBJOB@?$CILjava?1lang?1Object?$DL?$CJLjava?1lang?1@ 0000000140003310     exeCallerAccessTest.obj
 0002:00000338       ??_C@_03HNAFFKGA@get@      0000000140003338     exeCallerAccessTest.obj
 0002:00000340       ??_C@_0BG@DHOOFEJE@?$CILjava?1lang?1Object?$DL?$CJZ@ 0000000140003340     exeCallerAccessTest.obj
 0002:00000358       ??_C@_09EEAPPKDN@canAccess@ 0000000140003358     exeCallerAccessTest.obj
 0002:00000364       ??_C@_04LHKBAEFM@?$CIZ?$CJV@ 0000000140003364     exeCallerAccessTest.obj
 0002:00000370       ??_C@_0O@FAFFJLEJ@setAccessible@ 0000000140003370     exeCallerAccessTest.obj
 0002:00000380       ??_C@_03MMPFGPID@?$CI?$CJZ@ 0000000140003380     exeCallerAccessTest.obj
 0002:00000388       ??_C@_0BB@LKDBNJOO@trySetAccessible@ 0000000140003388     exeCallerAccessTest.obj
 0002:0000039c       ??_C@_04KDPJLEDB@TYPE@     000000014000339c     exeCallerAccessTest.obj
 0002:000003a8       ??_C@_0BC@GNOOPENL@java?4lang?4Integer@ 00000001400033a8     exeCallerAccessTest.obj
 0002:000003c0       ??_C@_0CP@GLPKDNMH@ERROR?3?5fail?5to?5access?5java?4lang@ 00000001400033c0     exeCallerAccessTest.obj
 0002:000003f0       ??_C@_0BF@BBLEIMJC@INVALID_FIELD_OFFSET@ 00000001400033f0     exeCallerAccessTest.obj
 0002:00000408       ??_C@_0BJ@MBHLIICD@jdk?4internal?4misc?4Unsafe@ 0000000140003408     exeCallerAccessTest.obj
 0002:00000428       ??_C@_0BH@CDDANCFJ@ERROR?3?5IAE?5not?5thrown?6@ 0000000140003428     exeCallerAccessTest.obj
 0002:00000440       ??_C@_0CM@HGHELFND@ERROR?3?5exception?5is?5not?5an?5inst@ 0000000140003440     exeCallerAccessTest.obj
 0002:0000046c       ??_C@_06EKOLBGFH@PUBLIC@   000000014000346c     exeCallerAccessTest.obj
 0002:00000478       ??_C@_0BL@NNIKOAFH@java?4lang?4reflect?4Modifier@ 0000000140003478     exeCallerAccessTest.obj
 0002:000004a0       ??_C@_0EK@DINAAAMK@ERROR?3?5unexpected?5result?5from?5t@ 00000001400034a0     exeCallerAccessTest.obj
 0002:000004f0       ??_C@_0EH@OPNGIGOK@ERROR?3?5unexpected?5result?5from?5t@ 00000001400034f0     exeCallerAccessTest.obj
 0002:00000540       __xmm@ffffffffffffffffffffffffffffffff 0000000140003540     MSVCRT:utility.obj
 0002:00000550       _load_config_used          0000000140003550     MSVCRT:loadcfg.obj
 0002:00000700       __volatile_metadata        0000000140003700     <linker-defined>
 0002:00000a10       __rtc_iaa                  0000000140003a10     MSVCRT:initsect.obj
 0002:00000a18       __rtc_izz                  0000000140003a18     MSVCRT:initsect.obj
 0002:00000a20       __rtc_taa                  0000000140003a20     MSVCRT:initsect.obj
 0002:00000a28       __rtc_tzz                  0000000140003a28     MSVCRT:initsect.obj
 0002:00000b34       __IMPORT_DESCRIPTOR_jvm    0000000140003b34     jvm:jvm.dll
 0002:00000b48       __IMPORT_DESCRIPTOR_KERNEL32 0000000140003b48     kernel32:KERNEL32.dll
 0002:00000b5c       __IMPORT_DESCRIPTOR_VCRUNTIME140 0000000140003b5c     vcruntime:VCRUNTIME140.dll
 0002:00000b70       __IMPORT_DESCRIPTOR_api-ms-win-crt-stdio-l1-1-0 0000000140003b70     ucrt:api-ms-win-crt-stdio-l1-1-0.dll
 0002:00000b84       __IMPORT_DESCRIPTOR_api-ms-win-crt-runtime-l1-1-0 0000000140003b84     ucrt:api-ms-win-crt-runtime-l1-1-0.dll
 0002:00000b98       __IMPORT_DESCRIPTOR_api-ms-win-crt-math-l1-1-0 0000000140003b98     ucrt:api-ms-win-crt-math-l1-1-0.dll
 0002:00000bac       __IMPORT_DESCRIPTOR_api-ms-win-crt-locale-l1-1-0 0000000140003bac     ucrt:api-ms-win-crt-locale-l1-1-0.dll
 0002:00000bc0       __IMPORT_DESCRIPTOR_api-ms-win-crt-heap-l1-1-0 0000000140003bc0     ucrt:api-ms-win-crt-heap-l1-1-0.dll
 0002:00000bd4       __NULL_IMPORT_DESCRIPTOR   0000000140003bd4     jvm:jvm.dll
 0003:00000000       __scrt_native_dllmain_reason 0000000140005000     MSVCRT:utility.obj
 0003:00000004       __scrt_default_matherr     0000000140005004     MSVCRT:matherr.obj
 0003:00000008       __isa_available            0000000140005008     MSVCRT:cpu_disp.obj
 0003:0000000c       __isa_enabled              000000014000500c     MSVCRT:cpu_disp.obj
 0003:00000010       __memset_fast_string_threshold 0000000140005010     MSVCRT:cpu_disp.obj
 0003:00000018       __memset_nt_threshold      0000000140005018     MSVCRT:cpu_disp.obj
 0003:00000020       __security_cookie          0000000140005020     MSVCRT:gs_cookie.obj
 0003:00000028       __security_cookie_complement 0000000140005028     MSVCRT:gs_cookie.obj
 0003:00000030       __scrt_ucrt_dll_is_in_use  0000000140005030     MSVCRT:ucrt_stubs.obj
 0003:00000080       __scrt_current_native_startup_state 0000000140005080     MSVCRT:utility.obj
 0003:00000088       __scrt_native_startup_lock 0000000140005088     MSVCRT:utility.obj
 0003:000000d0       ?__type_info_root_node@@3U__type_info_node@@A 00000001400050d0     MSVCRT:tncleanup.obj
 0003:000000e0       ?_OptionsStorage@?1??__local_stdio_scanf_options@@9@4_KA 00000001400050e0     MSVCRT:default_local_stdio_options.obj
 0003:000000e8       __scrt_debugger_hook_flag  00000001400050e8     MSVCRT:utility_desktop.obj
 0003:000000ec       __favor                    00000001400050ec     MSVCRT:cpu_disp.obj
 0003:000000f0       ?_OptionsStorage@?1??__local_stdio_printf_options@@9@9 00000001400050f0     <common>
 0003:000000f8       __dyn_tls_dtor_callback    00000001400050f8     <common>
 0003:00000100       __dyn_tls_init_callback    0000000140005100     <common>

 entry point at        0001:00000a28

 Static symbols

 0000:ffff8000       .debug$S                   0000000140000000     vcruntime:VCRUNTIME140.dll
 0000:ffff8000       .debug$S                   0000000140000000     vcruntime:VCRUNTIME140.dll
 0000:ffff8000       .debug$S                   0000000140000000     vcruntime:VCRUNTIME140.dll
 0000:ffff8000       .debug$S                   0000000140000000     vcruntime:VCRUNTIME140.dll
 0000:ffff8000       .debug$S                   0000000140000000     vcruntime:VCRUNTIME140.dll
 0000:ffff8000       .debug$S                   0000000140000000     vcruntime:VCRUNTIME140.dll
 0000:ffff8000       .debug$S                   0000000140000000     ucrt:api-ms-win-crt-heap-l1-1-0.dll
 0000:ffff8000       .debug$S                   0000000140000000     ucrt:api-ms-win-crt-locale-l1-1-0.dll
 0000:ffff8000       .debug$S                   0000000140000000     ucrt:api-ms-win-crt-math-l1-1-0.dll
 0000:ffff8000       .debug$S                   0000000140000000     ucrt:api-ms-win-crt-runtime-l1-1-0.dll
 0000:ffff8000       .debug$S                   0000000140000000     ucrt:api-ms-win-crt-runtime-l1-1-0.dll
 0000:ffff8000       .debug$S                   0000000140000000     ucrt:api-ms-win-crt-runtime-l1-1-0.dll
 0000:ffff8000       .debug$S                   0000000140000000     ucrt:api-ms-win-crt-runtime-l1-1-0.dll
 0000:ffff8000       .debug$S                   0000000140000000     ucrt:api-ms-win-crt-runtime-l1-1-0.dll
 0000:ffff8000       .debug$S                   0000000140000000     ucrt:api-ms-win-crt-runtime-l1-1-0.dll
 0000:ffff8000       .debug$S                   0000000140000000     ucrt:api-ms-win-crt-runtime-l1-1-0.dll
 0000:ffff8000       .debug$S                   0000000140000000     ucrt:api-ms-win-crt-runtime-l1-1-0.dll
 0000:ffff8000       .debug$S                   0000000140000000     ucrt:api-ms-win-crt-runtime-l1-1-0.dll
 0000:ffff8000       .debug$S                   0000000140000000     ucrt:api-ms-win-crt-runtime-l1-1-0.dll
 0000:ffff8000       .debug$S                   0000000140000000     ucrt:api-ms-win-crt-runtime-l1-1-0.dll
 0000:ffff8000       .debug$S                   0000000140000000     ucrt:api-ms-win-crt-runtime-l1-1-0.dll
 0000:ffff8000       .debug$S                   0000000140000000     ucrt:api-ms-win-crt-runtime-l1-1-0.dll
 0000:ffff8000       .debug$S                   0000000140000000     ucrt:api-ms-win-crt-runtime-l1-1-0.dll
 0000:ffff8000       .debug$S                   0000000140000000     ucrt:api-ms-win-crt-runtime-l1-1-0.dll
 0000:ffff8000       .debug$S                   0000000140000000     ucrt:api-ms-win-crt-runtime-l1-1-0.dll
 0000:ffff8000       .debug$S                   0000000140000000     ucrt:api-ms-win-crt-runtime-l1-1-0.dll
 0000:ffff8000       .debug$S                   0000000140000000     ucrt:api-ms-win-crt-runtime-l1-1-0.dll
 0000:ffff8000       .debug$S                   0000000140000000     ucrt:api-ms-win-crt-runtime-l1-1-0.dll
 0000:ffff8000       .debug$S                   0000000140000000     ucrt:api-ms-win-crt-runtime-l1-1-0.dll
 0000:ffff8000       .debug$S                   0000000140000000     ucrt:api-ms-win-crt-runtime-l1-1-0.dll
 0000:ffff8000       .debug$S                   0000000140000000     ucrt:api-ms-win-crt-stdio-l1-1-0.dll
 0000:ffff8000       .debug$S                   0000000140000000     ucrt:api-ms-win-crt-stdio-l1-1-0.dll
 0000:ffff8000       .debug$S                   0000000140000000     ucrt:api-ms-win-crt-stdio-l1-1-0.dll
 0000:ffff8000       .debug$S                   0000000140000000     ucrt:api-ms-win-crt-stdio-l1-1-0.dll
 0000:ffff8000       .debug$S                   0000000140000000     kernel32:KERNEL32.dll
 0000:ffff8000       .debug$S                   0000000140000000     kernel32:KERNEL32.dll
 0000:ffff8000       .debug$S                   0000000140000000     kernel32:KERNEL32.dll
 0000:ffff8000       .debug$S                   0000000140000000     kernel32:KERNEL32.dll
 0000:ffff8000       .debug$S                   0000000140000000     kernel32:KERNEL32.dll
 0000:ffff8000       .debug$S                   0000000140000000     kernel32:KERNEL32.dll
 0000:ffff8000       .debug$S                   0000000140000000     kernel32:KERNEL32.dll
 0000:ffff8000       .debug$S                   0000000140000000     kernel32:KERNEL32.dll
 0000:ffff8000       .debug$S                   0000000140000000     kernel32:KERNEL32.dll
 0000:ffff8000       .debug$S                   0000000140000000     kernel32:KERNEL32.dll
 0000:ffff8000       .debug$S                   0000000140000000     kernel32:KERNEL32.dll
 0000:ffff8000       .debug$S                   0000000140000000     kernel32:KERNEL32.dll
 0000:ffff8000       .debug$S                   0000000140000000     kernel32:KERNEL32.dll
 0000:ffff8000       .debug$S                   0000000140000000     kernel32:KERNEL32.dll
 0000:ffff8000       .debug$S                   0000000140000000     jvm:jvm.dll
 0001:000002b0       run                        00000001400012b0 f   exeCallerAccessTest.obj
 0001:000007c8       ?pre_c_initialization@@YAHXZ 00000001400017c8 f   MSVCRT:exe_main.obj
 0001:00000880       ?post_pgo_initialization@@YAHXZ 0000000140001880 f   MSVCRT:exe_main.obj
 0001:00000890       ?pre_cpp_initialization@@YAXXZ 0000000140001890 f   MSVCRT:exe_main.obj
 0001:000008ac       ?__scrt_common_main_seh@@YAHXZ 00000001400018ac f   MSVCRT:exe_main.obj
 0001:000012a0       $$000000                   00000001400022a0     MSVCRT:guard_dispatch.obj
 0001:000012c0       $$000000                   00000001400022c0     MSVCRT:guard_xfg_dispatch.obj
 0001:000012d6       ?filt$0@?0??__scrt_common_main_seh@@YAHXZ@4HA 00000001400022d6 f   MSVCRT:exe_main.obj
 0001:000012f4       __scrt_is_nonwritable_in_current_image$filt$0 00000001400022f4 f   MSVCRT:utility.obj
 0002:000001e0       ?pre_cpp_initializer@@3P6AXXZEA 00000001400031e0     MSVCRT:exe_main.obj
 0002:000001f8       ?pre_c_initializer@@3P6AHXZEA 00000001400031f8     MSVCRT:exe_main.obj
 0002:00000200       ?post_pgo_initializer@@3P6AHXZEA 0000000140003200     MSVCRT:exe_main.obj
 0002:00000a30       $unwind$printf             0000000140003a30     exeCallerAccessTest.obj
 0002:00000a3c       $unwind$getField           0000000140003a3c     exeCallerAccessTest.obj
 0002:00000a3c       $unwind$setAccessible      0000000140003a3c     exeCallerAccessTest.obj
 0002:00000a50       $unwind$checkAndClearIllegalAccessExceptionThrown 0000000140003a50     exeCallerAccessTest.obj
 0002:00000a50       $unwind$?pre_c_initialization@@YAHXZ 0000000140003a50     MSVCRT:exe_main.obj
 0002:00000a50       $unwind$__scrt_initialize_crt 0000000140003a50     MSVCRT:utility.obj
 0002:00000a50       $unwind$__scrt_initialize_onexit_tables 0000000140003a50     MSVCRT:utility.obj
 0002:00000a50       $unwind$__scrt_release_startup_lock 0000000140003a50     MSVCRT:utility.obj
 0002:00000a50       $unwind$__scrt_uninitialize_crt 0000000140003a50     MSVCRT:utility.obj
 0002:00000a50       $unwind$_onexit            0000000140003a50     MSVCRT:utility.obj
 0002:00000a58       $unwind$checkAccess        0000000140003a58     exeCallerAccessTest.obj
 0002:00000a58       $unwind$trySetAccessible   0000000140003a58     exeCallerAccessTest.obj
 0002:00000a70       $unwind$run                0000000140003a70     exeCallerAccessTest.obj
 0002:00000a80       $unwind$main               0000000140003a80     exeCallerAccessTest.obj
 0002:00000a80       $unwind$__scrt_initialize_default_local_stdio_options 0000000140003a80     MSVCRT:default_local_stdio_options.obj
 0002:00000a80       $unwind$?post_pgo_initialization@@YAHXZ 0000000140003a80     MSVCRT:exe_main.obj
 0002:00000a80       $unwind$?pre_cpp_initialization@@YAXXZ 0000000140003a80     MSVCRT:exe_main.obj
 0002:00000a80       $unwind$mainCRTStartup     0000000140003a80     MSVCRT:exe_main.obj
 0002:00000a80       $unwind$__scrt_acquire_startup_lock 0000000140003a80     MSVCRT:utility.obj
 0002:00000a80       $unwind$atexit             0000000140003a80     MSVCRT:utility.obj
 0002:00000a80       $unwind$__scrt_is_managed_app 0000000140003a80     MSVCRT:utility_desktop.obj
 0002:00000a88       $unwind$?__scrt_common_main_seh@@YAHXZ 0000000140003a88     MSVCRT:exe_main.obj
 0002:00000ac0       $unwind$?filt$0@?0??__scrt_common_main_seh@@YAHXZ@4HA 0000000140003ac0     MSVCRT:exe_main.obj
 0002:00000ac8       $unwind$__scrt_is_nonwritable_in_current_image 0000000140003ac8     MSVCRT:utility.obj
 0002:00000ae8       $unwind$__scrt_is_nonwritable_in_current_image$filt$0 0000000140003ae8     MSVCRT:utility.obj
 0002:00000af0       $unwind$__security_init_cookie 0000000140003af0     MSVCRT:gs_support.obj
 0002:00000afc       $unwind$__scrt_fastfail    0000000140003afc     MSVCRT:utility_desktop.obj
 0002:00000b0c       $unwind$_RTC_Initialize    0000000140003b0c     MSVCRT:initsect.obj
 0002:00000b0c       $unwind$_RTC_Terminate     0000000140003b0c     MSVCRT:initsect.obj
 0002:00000b0c       $unwind$__scrt_unhandled_exception_filter 0000000140003b0c     MSVCRT:utility_desktop.obj
 0002:00000b18       $unwind$__isa_available_init 0000000140003b18     MSVCRT:cpu_disp.obj
 0002:00000b28       $xdatasym                  0000000140003b28     MSVCRT:guard_dispatch.obj
 0002:00000b30       $xdatasym                  0000000140003b30     MSVCRT:guard_xfg_dispatch.obj
 0002:00000d9c       .idata$6                   0000000140003d9c     jvm:jvm.dll
 0002:00000eda       .idata$6                   0000000140003eda     kernel32:KERNEL32.dll
 0002:00000f3e       .idata$6                   0000000140003f3e     vcruntime:VCRUNTIME140.dll
 0002:0000112e       .idata$6                   000000014000412e     ucrt:api-ms-win-crt-stdio-l1-1-0.dll
 0002:0000114e       .idata$6                   000000014000414e     ucrt:api-ms-win-crt-runtime-l1-1-0.dll
 0002:00001170       .idata$6                   0000000140004170     ucrt:api-ms-win-crt-math-l1-1-0.dll
 0002:00001190       .idata$6                   0000000140004190     ucrt:api-ms-win-crt-locale-l1-1-0.dll
 0002:000011b2       .idata$6                   00000001400041b2     ucrt:api-ms-win-crt-heap-l1-1-0.dll
 0003:00000040       classClass                 0000000140005040     exeCallerAccessTest.obj
 0003:00000048       iaeClass                   0000000140005048     exeCallerAccessTest.obj
 0003:00000050       mid_Class_forName          0000000140005050     exeCallerAccessTest.obj
 0003:00000058       mid_Class_getField         0000000140005058     exeCallerAccessTest.obj
 0003:00000060       mid_Field_get              0000000140005060     exeCallerAccessTest.obj
 0003:00000068       mid_Field_canAccess        0000000140005068     exeCallerAccessTest.obj
 0003:00000070       mid_Field_trySetAccessible 0000000140005070     exeCallerAccessTest.obj
 0003:00000078       mid_Field_setAccessible    0000000140005078     exeCallerAccessTest.obj
 0003:00000090       ?is_initialized_as_dll@@3_NA 0000000140005090     MSVCRT:utility.obj
 0003:00000091       ?module_local_atexit_table_initialized@@3_NA 0000000140005091     MSVCRT:utility.obj
 0003:00000098       ?module_local_atexit_table@@3U_onexit_table_t@@A 0000000140005098     MSVCRT:utility.obj
 0003:000000b0       ?module_local_at_quick_exit_table@@3U_onexit_table_t@@A 00000001400050b0     MSVCRT:utility.obj
